 getallstktr001

 Timestamp is c616bde3 (reproducible build file hash)

 Preferred load address is 0000000180000000

 Start         Length     Name                   Class
 0001:00000000 000030e0H .text$mn                CODE
 0001:000030e0 00000036H .text$mn$00             CODE
 0001:00003116 00000092H .text$x                 CODE
 0002:00000000 00000198H .idata$5                DATA
 0002:00000198 00000038H .00cfg                  DATA
 0002:000001d0 00000008H .CRT$XCA                DATA
 0002:000001d8 00000008H .CRT$XCZ                DATA
 0002:000001e0 00000008H .CRT$XIA                DATA
 0002:000001e8 00000008H .CRT$XIC                DATA
 0002:000001f0 00000008H .CRT$XIZ                DATA
 0002:000001f8 00000008H .CRT$XLA                DATA
 0002:00000200 00000008H .CRT$XLZ                DATA
 0002:00000208 00000008H .CRT$XPA                DATA
 0002:00000210 00000008H .CRT$XPZ                DATA
 0002:00000218 00000008H .CRT$XTA                DATA
 0002:00000220 00000010H .CRT$XTZ                DATA
 0002:00000228 00000000H .gehcont$y              DATA
 0002:00000228 00000000H .gfids$y                DATA
 0002:00000230 00001e50H .rdata                  DATA
 0002:00002080 00000000H .rdata$CastGuardVftablesA DATA
 0002:00002080 00000000H .rdata$CastGuardVftablesC DATA
 0002:00002080 00000028H .rdata$T                DATA
 0002:000020a8 000000a4H .rdata$voltmd           DATA
 0002:0000214c 0000031cH .rdata$zzzdbg           DATA
 0002:00002468 00000008H .rtc$IAA                DATA
 0002:00002470 00000008H .rtc$IZZ                DATA
 0002:00002478 00000008H .rtc$TAA                DATA
 0002:00002480 00000008H .rtc$TZZ                DATA
 0002:00002488 00000004H .tls                    DATA
 0002:0000248c 00000004H .tls$                   DATA
 0002:00002490 00000008H .tls$ZZZ                DATA
 0002:00002498 00000358H .xdata                  DATA
 0002:000027f0 00000680H .edata                  DATA
 0002:00002e70 00000064H .idata$2                DATA
 0002:00002ed4 00000014H .idata$3                DATA
 0002:00002ee8 00000198H .idata$4                DATA
 0002:00003080 0000041eH .idata$6                DATA
 0003:00000000 00000080H .data                   DATA
 0003:00000080 0001b278H .bss                    DATA
 0004:00000000 000003fcH .pdata                  DATA

  Address         Publics by Value              Rva+Base               Lib:Object

 0000:00000000       __AbsoluteZero             0000000000000000     <absolute>
 0000:00000000       ___safe_se_handler_count   0000000000000000     <absolute>
 0000:00000000       ___safe_se_handler_table   0000000000000000     <absolute>
 0000:00000000       __arm64x_extra_rfe_table   0000000000000000     <absolute>
 0000:00000000       __arm64x_extra_rfe_table_size 0000000000000000     <absolute>
 0000:00000000       __arm64x_native_entrypoint 0000000000000000     <absolute>
 0000:00000000       __arm64x_redirection_metadata 0000000000000000     <absolute>
 0000:00000000       __arm64x_redirection_metadata_count 0000000000000000     <absolute>
 0000:00000000       __dynamic_value_reloc_table 0000000000000000     <absolute>
 0000:00000000       __enclave_config           0000000000000000     <absolute>
 0000:00000000       __guard_check_icall_a64n_fptr 0000000000000000     <absolute>
 0000:00000000       __guard_eh_cont_count      0000000000000000     <absolute>
 0000:00000000       __guard_eh_cont_table      0000000000000000     <absolute>
 0000:00000000       __guard_fids_count         0000000000000000     <absolute>
 0000:00000000       __guard_fids_table         0000000000000000     <absolute>
 0000:00000000       __guard_iat_count          0000000000000000     <absolute>
 0000:00000000       __guard_iat_table          0000000000000000     <absolute>
 0000:00000000       __guard_longjmp_count      0000000000000000     <absolute>
 0000:00000000       __guard_longjmp_table      0000000000000000     <absolute>
 0000:00000000       __hybrid_auxiliary_iat     0000000000000000     <absolute>
 0000:00000000       __hybrid_auxiliary_iat_copy 0000000000000000     <absolute>
 0000:00000000       __hybrid_code_map          0000000000000000     <absolute>
 0000:00000000       __hybrid_code_map_count    0000000000000000     <absolute>
 0000:00000000       __x64_code_ranges_to_entry_points 0000000000000000     <absolute>
 0000:00000000       __x64_code_ranges_to_entry_points_count 0000000000000000     <absolute>
 0000:00000100       __guard_flags              0000000000000100     <absolute>
 0000:00000000       __ImageBase                0000000180000000     <linker-defined>
 0001:00000000       ?NewObject@JNIEnv_@@QEAAPEAV_jobject@@PEAV_jclass@@PEAU_jmethodID@@ZZ 0000000180001000 f i libgetallstktr001.obj
 0001:00000028       ?TranslateError@@YAPEBDW4jvmtiError@@@Z 0000000180001028 f   libgetallstktr001.obj
 0001:000002e0       ?nsk_jni_check_exception@@YAHPEAUJNIEnv_@@QEBDH@Z 00000001800012e0 f   libgetallstktr001.obj
 0001:00000424       ?nsk_jni_lverify@@YAHHPEAUJNIEnv_@@HQEBDH1ZZ 0000000180001424 f   libgetallstktr001.obj
 0001:000004c4       Agent_Initialize           00000001800014c4 f   libgetallstktr001.obj
 0001:00000558       Agent_OnAttach             0000000180001558 f   libgetallstktr001.obj
 0001:00000558       Agent_OnLoad               0000000180001558 f   libgetallstktr001.obj
 0001:00000560       Java_nsk_jvmti_unit_FollowReferences_FollowRefObjects_addRefToVerify 0000000180001560 f   libgetallstktr001.obj
 0001:00000738       Java_nsk_jvmti_unit_FollowReferences_FollowRefObjects_getTag 0000000180001738 f   libgetallstktr001.obj
 0001:000007f8       Java_nsk_jvmti_unit_FollowReferences_FollowRefObjects_resetRefsToVerify 00000001800017f8 f   libgetallstktr001.obj
 0001:00000800       Java_nsk_jvmti_unit_FollowReferences_FollowRefObjects_resetTags 0000000180001800 f   libgetallstktr001.obj
 0001:00000844       Java_nsk_jvmti_unit_FollowReferences_FollowRefObjects_setTag 0000000180001844 f   libgetallstktr001.obj
 0001:00000a9c       Java_nsk_jvmti_unit_GetAllStackTraces_getallstktr001_CompareStackTraces 0000000180001a9c f   libgetallstktr001.obj
 0001:00000abc       Java_nsk_jvmti_unit_GetAllStackTraces_getallstktr001_CreateRawMonitor 0000000180001abc f   libgetallstktr001.obj
 0001:00000b40       Java_nsk_jvmti_unit_GetAllStackTraces_getallstktr001_DeallocateBuffers 0000000180001b40 f   libgetallstktr001.obj
 0001:00000c28       Java_nsk_jvmti_unit_GetAllStackTraces_getallstktr001_ForceGC 0000000180001c28 f   libgetallstktr001.obj
 0001:00000c60       Java_nsk_jvmti_unit_GetAllStackTraces_getallstktr001_GetAllStackTraces 0000000180001c60 f   libgetallstktr001.obj
 0001:00000d58       Java_nsk_jvmti_unit_GetAllStackTraces_getallstktr001_GetResult 0000000180001d58 f   libgetallstktr001.obj
 0001:00000d60       Java_nsk_jvmti_unit_GetAllStackTraces_getallstktr001_GetThreadListStackTraces 0000000180001d60 f   libgetallstktr001.obj
 0001:00000db8       Java_nsk_jvmti_unit_GetAllStackTraces_getallstktr001_GetThreadsInfo 0000000180001db8 f   libgetallstktr001.obj
 0001:00000ea0       Java_nsk_jvmti_unit_GetAllStackTraces_getallstktr001_RawMonitorEnter 0000000180001ea0 f   libgetallstktr001.obj
 0001:00000ee0       Java_nsk_jvmti_unit_GetAllStackTraces_getallstktr001_RawMonitorExit 0000000180001ee0 f   libgetallstktr001.obj
 0001:00000f20       Java_nsk_share_jvmti_ArgumentHandler_getAgentOptionsString 0000000180001f20 f   libgetallstktr001.obj
 0001:00000fd0       Java_nsk_share_jvmti_DebugeeClass_checkStatus 0000000180001fd0 f   libgetallstktr001.obj
 0001:00001058       Java_nsk_share_jvmti_DebugeeClass_resetAgentData 0000000180002058 f   libgetallstktr001.obj
 0001:000010b8       Java_nsk_share_jvmti_RedefineAgent_agentStatus 00000001800020b8 f   libgetallstktr001.obj
 0001:000010c4       Java_nsk_share_jvmti_RedefineAgent_isRedefined 00000001800020c4 f   libgetallstktr001.obj
 0001:000010d0       Java_nsk_share_jvmti_RedefineAgent_redefineAttempted 00000001800020d0 f   libgetallstktr001.obj
 0001:000010dc       MA_checkStatus             00000001800020dc f   libgetallstktr001.obj
 0001:00001180       __local_stdio_printf_options 0000000180002180 f i libgetallstktr001.obj
 0001:00001188       _snprintf                  0000000180002188 f i libgetallstktr001.obj
 0001:000013b8       compare_all_frames         00000001800023b8 f   libgetallstktr001.obj
 0001:00001464       compare_all_stack_traces   0000000180002464 f   libgetallstktr001.obj
 0001:000014cc       compare_one_stack_trace    00000001800024cc f   libgetallstktr001.obj
 0001:000015f0       exitOnError                00000001800025f0 f   libgetallstktr001.obj
 0001:000016a4       fprintf                    00000001800026a4 f i libgetallstktr001.obj
 0001:000016e8       nsk_jvmti_lverify          00000001800026e8 f   libgetallstktr001.obj
 0001:000017d8       nsk_jvmti_resetAgentData   00000001800027d8 f   libgetallstktr001.obj
 0001:00001858       nsk_jvmti_setFailStatus    0000000180002858 f   libgetallstktr001.obj
 0001:00001894       nsk_lcomplain              0000000180002894 f   libgetallstktr001.obj
 0001:000018b4       nsk_ldisplay               00000001800028b4 f   libgetallstktr001.obj
 0001:000018d4       nsk_ltrace                 00000001800028d4 f   libgetallstktr001.obj
 0001:000018f4       nsk_lvcomplain             00000001800028f4 f   libgetallstktr001.obj
 0001:00001aac       nsk_lvdisplay              0000000180002aac f   libgetallstktr001.obj
 0001:00001af8       nsk_lverify                0000000180002af8 f   libgetallstktr001.obj
 0001:00001b54       nsk_lvtrace                0000000180002b54 f   libgetallstktr001.obj
 0001:00001bb4       nsk_printf                 0000000180002bb4 f   libgetallstktr001.obj
 0001:00001bdc       nsk_vprintf                0000000180002bdc f   libgetallstktr001.obj
 0001:00001c90       printf                     0000000180002c90 f i libgetallstktr001.obj
 0001:000021b8       __raise_securityfailure    00000001800031b8 f   MSVCRT:gs_report.obj
 0001:000021ec       __report_gsfailure         00000001800031ec f   MSVCRT:gs_report.obj
 0001:0000242c       __GSHandlerCheck           000000018000342c f   MSVCRT:gshandler.obj
 0001:0000244c       __GSHandlerCheckCommon     000000018000344c f   MSVCRT:gshandler.obj
 0001:000024c0       __security_check_cookie    00000001800034c0 f   MSVCRT:amdsecgs.obj
 0001:00002800       _DllMainCRTStartup         0000000180003800 f   MSVCRT:dll_dllmain.obj
 0001:00002840       __scrt_acquire_startup_lock 0000000180003840 f   MSVCRT:utility.obj
 0001:0000287c       __scrt_dllmain_after_initialize_c 000000018000387c f   MSVCRT:utility.obj
 0001:000028b0       __scrt_dllmain_before_initialize_c 00000001800038b0 f   MSVCRT:utility.obj
 0001:000028c8       __scrt_dllmain_crt_thread_attach 00000001800038c8 f   MSVCRT:utility.obj
 0001:000028f0       __scrt_dllmain_crt_thread_detach 00000001800038f0 f   MSVCRT:utility.obj
 0001:00002908       __scrt_dllmain_exception_filter 0000000180003908 f   MSVCRT:utility.obj
 0001:00002968       __scrt_dllmain_uninitialize_c 0000000180003968 f   MSVCRT:utility.obj
 0001:00002998       __scrt_dllmain_uninitialize_critical 0000000180003998 f   MSVCRT:utility.obj
 0001:000029ac       __scrt_initialize_crt      00000001800039ac f   MSVCRT:utility.obj
 0001:000029f8       __scrt_initialize_onexit_tables 00000001800039f8 f   MSVCRT:utility.obj
 0001:00002a84       __scrt_is_nonwritable_in_current_image 0000000180003a84 f   MSVCRT:utility.obj
 0001:00002b1c       __scrt_release_startup_lock 0000000180003b1c f   MSVCRT:utility.obj
 0001:00002b40       __scrt_uninitialize_crt    0000000180003b40 f   MSVCRT:utility.obj
 0001:00002b6c       _onexit                    0000000180003b6c f   MSVCRT:utility.obj
 0001:00002ba8       atexit                     0000000180003ba8 f   MSVCRT:utility.obj
 0001:00002bc0       __crt_debugger_hook        0000000180003bc0 f   MSVCRT:utility_desktop.obj
 0001:00002bc8       __scrt_fastfail            0000000180003bc8 f   MSVCRT:utility_desktop.obj
 0001:00002d14       _guard_check_icall_nop     0000000180003d14 f i MSVCRT:guard_support.obj
 0001:00002d18       __security_init_cookie     0000000180003d18 f   MSVCRT:gs_support.obj
 0001:00002dc4       DllMain                    0000000180003dc4 f   MSVCRT:dll_dllmain_stub.obj
 0001:00002de8       ?__scrt_initialize_type_info@@YAXXZ 0000000180003de8 f   MSVCRT:tncleanup.obj
 0001:00002df8       ?__scrt_uninitialize_type_info@@YAXXZ 0000000180003df8 f   MSVCRT:tncleanup.obj
 0001:00002e04       __local_stdio_scanf_options 0000000180003e04 f i MSVCRT:default_local_stdio_options.obj
 0001:00002e0c       __scrt_initialize_default_local_stdio_options 0000000180003e0c f   MSVCRT:default_local_stdio_options.obj
 0001:00002e28       __scrt_get_dyn_tls_init_callback 0000000180003e28 f   MSVCRT:dyn_tls_init.obj
 0001:00002e30       _RTC_Initialize            0000000180003e30 f   MSVCRT:initsect.obj
 0001:00002e6c       _RTC_Terminate             0000000180003e6c f   MSVCRT:initsect.obj
 0001:00002ea8       __isa_available_init       0000000180003ea8 f   MSVCRT:cpu_disp.obj
 0001:00003054       _get_startup_argv_mode     0000000180004054 f   MSVCRT:argv_mode.obj
 0001:0000305c       __scrt_is_ucrt_dll_in_use  000000018000405c f   MSVCRT:ucrt_detection.obj
 0001:00003070       memcpy                     0000000180004070 f   vcruntime:VCRUNTIME140.dll
 0001:00003076       memset                     0000000180004076 f   vcruntime:VCRUNTIME140.dll
 0001:0000307c       strchr                     000000018000407c f   vcruntime:VCRUNTIME140.dll
 0001:00003082       __C_specific_handler       0000000180004082 f   vcruntime:VCRUNTIME140.dll
 0001:00003088       __std_type_info_destroy_list 0000000180004088 f   vcruntime:VCRUNTIME140.dll
 0001:0000308e       strlen                     000000018000408e f   ucrt:api-ms-win-crt-string-l1-1-0.dll
 0001:00003094       _initterm                  0000000180004094 f   ucrt:api-ms-win-crt-runtime-l1-1-0.dll
 0001:0000309a       _initterm_e                000000018000409a f   ucrt:api-ms-win-crt-runtime-l1-1-0.dll
 0001:000030a0       _seh_filter_dll            00000001800040a0 f   ucrt:api-ms-win-crt-runtime-l1-1-0.dll
 0001:000030a6       _configure_narrow_argv     00000001800040a6 f   ucrt:api-ms-win-crt-runtime-l1-1-0.dll
 0001:000030ac       _initialize_narrow_environment 00000001800040ac f   ucrt:api-ms-win-crt-runtime-l1-1-0.dll
 0001:000030b2       _initialize_onexit_table   00000001800040b2 f   ucrt:api-ms-win-crt-runtime-l1-1-0.dll
 0001:000030b8       _register_onexit_function  00000001800040b8 f   ucrt:api-ms-win-crt-runtime-l1-1-0.dll
 0001:000030be       _execute_onexit_table      00000001800040be f   ucrt:api-ms-win-crt-runtime-l1-1-0.dll
 0001:000030c4       _crt_atexit                00000001800040c4 f   ucrt:api-ms-win-crt-runtime-l1-1-0.dll
 0001:000030ca       _cexit                     00000001800040ca f   ucrt:api-ms-win-crt-runtime-l1-1-0.dll
 0001:000030d0       __acrt_initialize          00000001800040d0 f   MSVCRT:ucrt_stubs.obj
 0001:000030d0       __acrt_thread_attach       00000001800040d0 f   MSVCRT:ucrt_stubs.obj
 0001:000030d0       __acrt_thread_detach       00000001800040d0 f   MSVCRT:ucrt_stubs.obj
 0001:000030d0       __acrt_uninitialize        00000001800040d0 f   MSVCRT:ucrt_stubs.obj
 0001:000030d0       __acrt_uninitialize_critical 00000001800040d0 f   MSVCRT:ucrt_stubs.obj
 0001:000030d0       __scrt_stub_for_acrt_initialize 00000001800040d0 f   MSVCRT:ucrt_stubs.obj
 0001:000030d0       __scrt_stub_for_acrt_thread_attach 00000001800040d0 f   MSVCRT:ucrt_stubs.obj
 0001:000030d0       __scrt_stub_for_acrt_thread_detach 00000001800040d0 f   MSVCRT:ucrt_stubs.obj
 0001:000030d0       __scrt_stub_for_acrt_uninitialize 00000001800040d0 f   MSVCRT:ucrt_stubs.obj
 0001:000030d0       __scrt_stub_for_acrt_uninitialize_critical 00000001800040d0 f   MSVCRT:ucrt_stubs.obj
 0001:000030d0       __vcrt_initialize          00000001800040d0 f   MSVCRT:ucrt_stubs.obj
 0001:000030d0       __vcrt_thread_attach       00000001800040d0 f   MSVCRT:ucrt_stubs.obj
 0001:000030d0       __vcrt_thread_detach       00000001800040d0 f   MSVCRT:ucrt_stubs.obj
 0001:000030d0       __vcrt_uninitialize        00000001800040d0 f   MSVCRT:ucrt_stubs.obj
 0001:000030d0       __vcrt_uninitialize_critical 00000001800040d0 f   MSVCRT:ucrt_stubs.obj
 0001:000030d4       __scrt_stub_for_is_c_termination_complete 00000001800040d4 f   MSVCRT:ucrt_stubs.obj
 0001:000030d4       _is_c_termination_complete 00000001800040d4 f   MSVCRT:ucrt_stubs.obj
 0001:000030f0       _guard_dispatch_icall_nop  00000001800040f0 f   MSVCRT:guard_dispatch.obj
 0001:00003110       _guard_xfg_dispatch_icall_nop 0000000180004110 f   MSVCRT:guard_xfg_dispatch.obj
 0002:00000000       __imp_RtlCaptureContext    0000000180005000     kernel32:KERNEL32.dll
 0002:00000008       __imp_RtlLookupFunctionEntry 0000000180005008     kernel32:KERNEL32.dll
 0002:00000010       __imp_RtlVirtualUnwind     0000000180005010     kernel32:KERNEL32.dll
 0002:00000018       __imp_UnhandledExceptionFilter 0000000180005018     kernel32:KERNEL32.dll
 0002:00000020       __imp_SetUnhandledExceptionFilter 0000000180005020     kernel32:KERNEL32.dll
 0002:00000028       __imp_GetCurrentProcess    0000000180005028     kernel32:KERNEL32.dll
 0002:00000030       __imp_TerminateProcess     0000000180005030     kernel32:KERNEL32.dll
 0002:00000038       __imp_IsProcessorFeaturePresent 0000000180005038     kernel32:KERNEL32.dll
 0002:00000040       __imp_CloseHandle          0000000180005040     kernel32:KERNEL32.dll
 0002:00000048       __imp_InitializeCriticalSectionAndSpinCount 0000000180005048     kernel32:KERNEL32.dll
 0002:00000050       __imp_DeleteCriticalSection 0000000180005050     kernel32:KERNEL32.dll
 0002:00000058       __imp_CreateEventW         0000000180005058     kernel32:KERNEL32.dll
 0002:00000060       __imp_GetModuleHandleW     0000000180005060     kernel32:KERNEL32.dll
 0002:00000068       __imp_GetProcAddress       0000000180005068     kernel32:KERNEL32.dll
 0002:00000070       __imp_IsDebuggerPresent    0000000180005070     kernel32:KERNEL32.dll
 0002:00000078       __imp_QueryPerformanceCounter 0000000180005078     kernel32:KERNEL32.dll
 0002:00000080       __imp_GetCurrentProcessId  0000000180005080     kernel32:KERNEL32.dll
 0002:00000088       __imp_GetCurrentThreadId   0000000180005088     kernel32:KERNEL32.dll
 0002:00000090       __imp_GetSystemTimeAsFileTime 0000000180005090     kernel32:KERNEL32.dll
 0002:00000098       __imp_DisableThreadLibraryCalls 0000000180005098     kernel32:KERNEL32.dll
 0002:000000a0       __imp_InitializeSListHead  00000001800050a0     kernel32:KERNEL32.dll
 0002:000000a8       \177KERNEL32_NULL_THUNK_DATA 00000001800050a8     kernel32:KERNEL32.dll
 0002:000000b0       __imp_memcpy               00000001800050b0     vcruntime:VCRUNTIME140.dll
 0002:000000b8       __imp_memset               00000001800050b8     vcruntime:VCRUNTIME140.dll
 0002:000000c0       __imp_strchr               00000001800050c0     vcruntime:VCRUNTIME140.dll
 0002:000000c8       __imp___C_specific_handler 00000001800050c8     vcruntime:VCRUNTIME140.dll
 0002:000000d0       __imp___std_type_info_destroy_list 00000001800050d0     vcruntime:VCRUNTIME140.dll
 0002:000000d8       \177VCRUNTIME140_NULL_THUNK_DATA 00000001800050d8     vcruntime:VCRUNTIME140.dll
 0002:000000e0       __imp__errno               00000001800050e0     ucrt:api-ms-win-crt-runtime-l1-1-0.dll
 0002:000000e8       __imp_exit                 00000001800050e8     ucrt:api-ms-win-crt-runtime-l1-1-0.dll
 0002:000000f0       __imp__cexit               00000001800050f0     ucrt:api-ms-win-crt-runtime-l1-1-0.dll
 0002:000000f8       __imp__crt_atexit          00000001800050f8     ucrt:api-ms-win-crt-runtime-l1-1-0.dll
 0002:00000100       __imp__execute_onexit_table 0000000180005100     ucrt:api-ms-win-crt-runtime-l1-1-0.dll
 0002:00000108       __imp__register_onexit_function 0000000180005108     ucrt:api-ms-win-crt-runtime-l1-1-0.dll
 0002:00000110       __imp__initialize_onexit_table 0000000180005110     ucrt:api-ms-win-crt-runtime-l1-1-0.dll
 0002:00000118       __imp__initialize_narrow_environment 0000000180005118     ucrt:api-ms-win-crt-runtime-l1-1-0.dll
 0002:00000120       __imp__configure_narrow_argv 0000000180005120     ucrt:api-ms-win-crt-runtime-l1-1-0.dll
 0002:00000128       __imp__seh_filter_dll      0000000180005128     ucrt:api-ms-win-crt-runtime-l1-1-0.dll
 0002:00000130       __imp__initterm_e          0000000180005130     ucrt:api-ms-win-crt-runtime-l1-1-0.dll
 0002:00000138       __imp__initterm            0000000180005138     ucrt:api-ms-win-crt-runtime-l1-1-0.dll
 0002:00000140       \177api-ms-win-crt-runtime-l1-1-0_NULL_THUNK_DATA 0000000180005140     ucrt:api-ms-win-crt-runtime-l1-1-0.dll
 0002:00000148       __imp___acrt_iob_func      0000000180005148     ucrt:api-ms-win-crt-stdio-l1-1-0.dll
 0002:00000150       __imp_fflush               0000000180005150     ucrt:api-ms-win-crt-stdio-l1-1-0.dll
 0002:00000158       __imp___stdio_common_vsprintf 0000000180005158     ucrt:api-ms-win-crt-stdio-l1-1-0.dll
 0002:00000160       __imp___stdio_common_vfprintf 0000000180005160     ucrt:api-ms-win-crt-stdio-l1-1-0.dll
 0002:00000168       \177api-ms-win-crt-stdio-l1-1-0_NULL_THUNK_DATA 0000000180005168     ucrt:api-ms-win-crt-stdio-l1-1-0.dll
 0002:00000170       __imp__strdup              0000000180005170     ucrt:api-ms-win-crt-string-l1-1-0.dll
 0002:00000170       __imp_strdup               0000000180005170     ucrt:api-ms-win-crt-string-l1-1-0.dll
 0002:00000178       __imp_strlen               0000000180005178     ucrt:api-ms-win-crt-string-l1-1-0.dll
 0002:00000180       __imp_strncmp              0000000180005180     ucrt:api-ms-win-crt-string-l1-1-0.dll
 0002:00000188       __imp_strncpy              0000000180005188     ucrt:api-ms-win-crt-string-l1-1-0.dll
 0002:00000190       \177api-ms-win-crt-string-l1-1-0_NULL_THUNK_DATA 0000000180005190     ucrt:api-ms-win-crt-string-l1-1-0.dll
 0002:00000198       __guard_check_icall_fptr   0000000180005198     MSVCRT:guard_support.obj
 0002:000001a0       __guard_xfg_check_icall_fptr 00000001800051a0     MSVCRT:guard_support.obj
 0002:000001a8       __guard_dispatch_icall_fptr 00000001800051a8     MSVCRT:guard_support.obj
 0002:000001b0       __guard_xfg_dispatch_icall_fptr 00000001800051b0     MSVCRT:guard_support.obj
 0002:000001b8       __guard_xfg_table_dispatch_icall_fptr 00000001800051b8     MSVCRT:guard_support.obj
 0002:000001c0       __castguard_check_failure_os_handled_fptr 00000001800051c0     MSVCRT:guard_support.obj
 0002:000001c8       __guard_memcpy_fptr        00000001800051c8     vcruntime:softmemtag.obj
 0002:000001d0       __xc_a                     00000001800051d0     MSVCRT:initializers.obj
 0002:000001d8       __xc_z                     00000001800051d8     MSVCRT:initializers.obj
 0002:000001e0       __xi_a                     00000001800051e0     MSVCRT:initializers.obj
 0002:000001f0       __xi_z                     00000001800051f0     MSVCRT:initializers.obj
 0002:000001f8       __xl_a                     00000001800051f8     MSVCRT:tlssup.obj
 0002:00000200       __xl_z                     0000000180005200     MSVCRT:tlssup.obj
 0002:00000208       __xp_a                     0000000180005208     MSVCRT:initializers.obj
 0002:00000210       __xp_z                     0000000180005210     MSVCRT:initializers.obj
 0002:00000218       __xt_a                     0000000180005218     MSVCRT:initializers.obj
 0002:00000220       __xt_z                     0000000180005220     MSVCRT:initializers.obj
 0002:00000230       g_refKindStr               0000000180005230     libgetallstktr001.obj
 0002:000003e0       ??_C@_09BPLDFGCI@unknown_0@ 00000001800053e0     libgetallstktr001.obj
 0002:000003f0       ??_C@_0BL@FPNMECJD@JVMTI_HEAP_REFERENCE_CLASS@ 00000001800053f0     libgetallstktr001.obj
 0002:00000410       ??_C@_0BL@FKGKKLNM@JVMTI_HEAP_REFERENCE_FIELD@ 0000000180005410     libgetallstktr001.obj
 0002:00000430       ??_C@_0CD@CAEHCFJF@JVMTI_HEAP_REFERENCE_ARRAY_ELEM@ 0000000180005430     libgetallstktr001.obj
 0002:00000458       ??_C@_0CC@DNEBMCNK@JVMTI_HEAP_REFERENCE_CLASS_LOAD@ 0000000180005458     libgetallstktr001.obj
 0002:00000480       ??_C@_0BN@CJMIPEBB@JVMTI_HEAP_REFERENCE_SIGNERS@ 0000000180005480     libgetallstktr001.obj
 0002:000004a0       ??_C@_0CH@HBOIDPEB@JVMTI_HEAP_REFERENCE_PROTECTION@ 00000001800054a0     libgetallstktr001.obj
 0002:000004c8       ??_C@_0BP@MDKGDGKL@JVMTI_HEAP_REFERENCE_INTERFACE@ 00000001800054c8     libgetallstktr001.obj
 0002:000004e8       ??_C@_0CC@JJMIHNJH@JVMTI_HEAP_REFERENCE_STATIC_FIE@ 00000001800054e8     libgetallstktr001.obj
 0002:00000510       ??_C@_0CD@IDHEEGID@JVMTI_HEAP_REFERENCE_CONSTANT_P@ 0000000180005510     libgetallstktr001.obj
 0002:00000538       ??_C@_0CA@EFFCHNG@JVMTI_HEAP_REFERENCE_SUPERCLASS@ 0000000180005538     libgetallstktr001.obj
 0002:00000558       ??_C@_0L@PCDFHGCJ@unknown_11@ 0000000180005558     libgetallstktr001.obj
 0002:00000568       ??_C@_0L@NJBICFOK@unknown_12@ 0000000180005568     libgetallstktr001.obj
 0002:00000578       ??_C@_0L@MAADBEKL@unknown_13@ 0000000180005578     libgetallstktr001.obj
 0002:00000588       ??_C@_0L@IPECICGM@unknown_14@ 0000000180005588     libgetallstktr001.obj
 0002:00000598       ??_C@_0L@JGFJLDCN@unknown_15@ 0000000180005598     libgetallstktr001.obj
 0002:000005a8       ??_C@_0L@LNHEOAOO@unknown_16@ 00000001800055a8     libgetallstktr001.obj
 0002:000005b8       ??_C@_0L@KEGPNBKP@unknown_17@ 00000001800055b8     libgetallstktr001.obj
 0002:000005c8       ??_C@_0L@CDPHMNGA@unknown_18@ 00000001800055c8     libgetallstktr001.obj
 0002:000005d8       ??_C@_0L@DKOMPMCB@unknown_19@ 00000001800055d8     libgetallstktr001.obj
 0002:000005e8       ??_C@_0L@OJGIPJDB@unknown_20@ 00000001800055e8     libgetallstktr001.obj
 0002:000005f8       ??_C@_0CA@KAOFNDEM@JVMTI_HEAP_REFERENCE_JNI_GLOBAL@ 00000001800055f8     libgetallstktr001.obj
 0002:00000618       ??_C@_0CC@HPFAJBK@JVMTI_HEAP_REFERENCE_SYSTEM_CLA@ 0000000180005618     libgetallstktr001.obj
 0002:00000640       ??_C@_0BN@FDEGFOHC@JVMTI_HEAP_REFERENCE_MONITOR@ 0000000180005640     libgetallstktr001.obj
 0002:00000660       ??_C@_0CB@HKIBCMAJ@JVMTI_HEAP_REFERENCE_STACK_LOCA@ 0000000180005660     libgetallstktr001.obj
 0002:00000688       ??_C@_0BP@EAACMMOE@JVMTI_HEAP_REFERENCE_JNI_LOCAL@ 0000000180005688     libgetallstktr001.obj
 0002:000006a8       ??_C@_0BM@IJDEOGOE@JVMTI_HEAP_REFERENCE_THREAD@ 00000001800056a8     libgetallstktr001.obj
 0002:000006c8       ??_C@_0BL@EDGPPKC@JVMTI_HEAP_REFERENCE_OTHER@ 00000001800056c8     libgetallstktr001.obj
 0002:000006e4       ??_C@_04BCJPDBDA@Code@     00000001800056e4     libgetallstktr001.obj
 0002:000006f0       ??_C@_0BA@OCLMCFKC@LineNumberTable@ 00000001800056f0     libgetallstktr001.obj
 0002:00000700       ??_C@_0BD@CPAEPILC@LocalVariableTable@ 0000000180005700     libgetallstktr001.obj
 0002:00000718       ??_C@_0BH@NMBDNHBD@LocalVariableTypeTable@ 0000000180005718     libgetallstktr001.obj
 0002:00000730       ??_C@_0O@HIHEEDNJ@StackMapTable@ 0000000180005730     libgetallstktr001.obj
 0002:00000740       ??_C@_0L@HCDIAMJG@?9?5?$CFs?0?5?$CFd?3?5@ 0000000180005740     libgetallstktr001.obj
 0002:00000750       ??_C@_0JI@HLPECLFI@?$CD?5?4?4?4?6?$CD?5ERROR?3?5too?5many?5complai@ 0000000180005750     libgetallstktr001.obj
 0002:000007f0       ??_C@_0ED@JNEKCCOB@The?5following?5fake?5exception?5st@ 00000001800057f0     libgetallstktr001.obj
 0002:00000838       ??_C@_0CN@FCNMDFBH@nsk?4share?4Fake_Exception_for_RU@ 0000000180005838     libgetallstktr001.obj
 0002:00000868       ??_C@_08PGFFNAEI@?$CI?$CFs?3?$CFd?$CJ?5@ 0000000180005868     libgetallstktr001.obj
 0002:00000878       ??_C@_0DP@IENMAEGI@s?2test?2hotspot?2jtreg?2vmTestbase@ 0000000180005878     libgetallstktr001.obj
 0002:000008b8       ??_C@_0BL@NDJLFFJB@?7at?5nsk_lvcomplain?$CI?$CFs?3?$CFd?$CJ?6@ 00000001800058b8     libgetallstktr001.obj
 0002:000008d8       ??_C@_0BC@JOOKAFKF@?$CD?5ERROR?3?5?$CFs?0?5?$CFd?3?5@ 00000001800058d8     libgetallstktr001.obj
 0002:000008f0       ??_C@_09KJEAHMEH@?$CD?5ERROR?3?5@ 00000001800058f0     libgetallstktr001.obj
 0002:000008fc       ??_C@_02GPIOPFAK@?$DO?$DO@ 00000001800058fc     libgetallstktr001.obj
 0002:00000900       ??_C@_02FODMEDOG@?$DM?$DM@ 0000000180005900     libgetallstktr001.obj
 0002:00000904       ??_C@_02DJGKEECL@?4?4@     0000000180005904     libgetallstktr001.obj
 0002:00000908       ??_C@_0O@CJPGJOAF@?9?5?$CFs?0?5?$CFd?3?5?$CFs?5@ 0000000180005908     libgetallstktr001.obj
 0002:00000918       ??_C@_0CB@IAKPDOIC@?$CD?5?5?5verified?5assertion?5is?5FALSE@ 0000000180005918     libgetallstktr001.obj
 0002:00000940       ??_C@_0CO@LGONDEPD@stdout?3?5fflush?5failed?5?9?5err?$DN?$CFd?5@ 0000000180005940     libgetallstktr001.obj
 0002:00000970       ??_C@_0CO@KBGKJPBD@stderr?3?5fflush?5failed?5?9?5err?$DN?$CFd?5@ 0000000180005970     libgetallstktr001.obj
 0002:000009a0       ??_C@_0BB@JCNMKLLK@JVMTI_ERROR_NONE@ 00000001800059a0     libgetallstktr001.obj
 0002:000009b8       ??_C@_0BL@LDIMKLPH@JVMTI_ERROR_INVALID_THREAD@ 00000001800059b8     libgetallstktr001.obj
 0002:000009d8       ??_C@_0CB@PJFPAIKJ@JVMTI_ERROR_INVALID_THREAD_GROU@ 00000001800059d8     libgetallstktr001.obj
 0002:00000a00       ??_C@_0BN@LLMKHMNF@JVMTI_ERROR_INVALID_PRIORITY@ 0000000180005a00     libgetallstktr001.obj
 0002:00000a20       ??_C@_0CB@MBOFKAGB@JVMTI_ERROR_THREAD_NOT_SUSPENDE@ 0000000180005a20     libgetallstktr001.obj
 0002:00000a48       ??_C@_0BN@FABOLPBI@JVMTI_ERROR_THREAD_SUSPENDED@ 0000000180005a48     libgetallstktr001.obj
 0002:00000a68       ??_C@_0BN@FDGNOBJM@JVMTI_ERROR_THREAD_NOT_ALIVE@ 0000000180005a68     libgetallstktr001.obj
 0002:00000a88       ??_C@_0BL@GOBIFKNJ@JVMTI_ERROR_INVALID_OBJECT@ 0000000180005a88     libgetallstktr001.obj
 0002:00000aa8       ??_C@_0BK@FCMAJPPC@JVMTI_ERROR_INVALID_CLASS@ 0000000180005aa8     libgetallstktr001.obj
 0002:00000ac8       ??_C@_0BP@IKLLBKEB@JVMTI_ERROR_CLASS_NOT_PREPARED@ 0000000180005ac8     libgetallstktr001.obj
 0002:00000ae8       ??_C@_0BN@KLPPLKG@JVMTI_ERROR_INVALID_METHODID@ 0000000180005ae8     libgetallstktr001.obj
 0002:00000b08       ??_C@_0BN@BCEKOKND@JVMTI_ERROR_INVALID_LOCATION@ 0000000180005b08     libgetallstktr001.obj
 0002:00000b28       ??_C@_0BM@DFDGPME@JVMTI_ERROR_INVALID_FIELDID@ 0000000180005b28     libgetallstktr001.obj
 0002:00000b48       ??_C@_0BL@NELIEPEC@JVMTI_ERROR_NO_MORE_FRAMES@ 0000000180005b48     libgetallstktr001.obj
 0002:00000b68       ??_C@_0BJ@BDBECFDM@JVMTI_ERROR_OPAQUE_FRAME@ 0000000180005b68     libgetallstktr001.obj
 0002:00000b88       ??_C@_0BK@MIIFNLOB@JVMTI_ERROR_TYPE_MISMATCH@ 0000000180005b88     libgetallstktr001.obj
 0002:00000ba8       ??_C@_0BJ@HPCAOILC@JVMTI_ERROR_INVALID_SLOT@ 0000000180005ba8     libgetallstktr001.obj
 0002:00000bc8       ??_C@_0BG@CHILOPNI@JVMTI_ERROR_DUPLICATE@ 0000000180005bc8     libgetallstktr001.obj
 0002:00000be0       ??_C@_0BG@DIEMLHKM@JVMTI_ERROR_NOT_FOUND@ 0000000180005be0     libgetallstktr001.obj
 0002:00000bf8       ??_C@_0BM@NHMCKHOB@JVMTI_ERROR_INVALID_MONITOR@ 0000000180005bf8     libgetallstktr001.obj
 0002:00000c18       ??_C@_0BO@PPEDAJGL@JVMTI_ERROR_NOT_MONITOR_OWNER@ 0000000180005c18     libgetallstktr001.obj
 0002:00000c38       ??_C@_0BG@FCAIPEID@JVMTI_ERROR_INTERRUPT@ 0000000180005c38     libgetallstktr001.obj
 0002:00000c50       ??_C@_0CB@EGDBNKOI@JVMTI_ERROR_INVALID_CLASS_FORMA@ 0000000180005c50     libgetallstktr001.obj
 0002:00000c78       ??_C@_0CG@DGKOGIAL@JVMTI_ERROR_CIRCULAR_CLASS_DEFI@ 0000000180005c78     libgetallstktr001.obj
 0002:00000ca0       ??_C@_0BP@ICEALPKC@JVMTI_ERROR_FAILS_VERIFICATION@ 0000000180005ca0     libgetallstktr001.obj
 0002:00000cc0       ??_C@_0DC@JDACLMIO@JVMTI_ERROR_UNSUPPORTED_REDEFIN@ 0000000180005cc0     libgetallstktr001.obj
 0002:00000cf8       ??_C@_0DE@GKDKNOMJ@JVMTI_ERROR_UNSUPPORTED_REDEFIN@ 0000000180005cf8     libgetallstktr001.obj
 0002:00000d30       ??_C@_0BO@LAFKIOG@JVMTI_ERROR_INVALID_TYPESTATE@ 0000000180005d30     libgetallstktr001.obj
 0002:00000d50       ??_C@_0DH@INDGCLLB@JVMTI_ERROR_UNSUPPORTED_REDEFIN@ 0000000180005d50     libgetallstktr001.obj
 0002:00000d88       ??_C@_0DE@NHEOMMGI@JVMTI_ERROR_UNSUPPORTED_REDEFIN@ 0000000180005d88     libgetallstktr001.obj
 0002:00000dc0       ??_C@_0CA@EKPNJOEP@JVMTI_ERROR_UNSUPPORTED_VERSION@ 0000000180005dc0     libgetallstktr001.obj
 0002:00000de0       ??_C@_0BN@OFFMAHHL@JVMTI_ERROR_NAMES_DONT_MATCH@ 0000000180005de0     libgetallstktr001.obj
 0002:00000e00       ??_C@_0DN@HHBBLAKE@JVMTI_ERROR_UNSUPPORTED_REDEFIN@ 0000000180005e00     libgetallstktr001.obj
 0002:00000e40       ??_C@_0DO@HMBGBGNA@JVMTI_ERROR_UNSUPPORTED_REDEFIN@ 0000000180005e40     libgetallstktr001.obj
 0002:00000e80       ??_C@_0BP@PBECGKHJ@JVMTI_ERROR_UNMODIFIABLE_CLASS@ 0000000180005e80     libgetallstktr001.obj
 0002:00000ea0       ??_C@_0BK@CANILEHF@JVMTI_ERROR_NOT_AVAILABLE@ 0000000180005ea0     libgetallstktr001.obj
 0002:00000ec0       ??_C@_0CE@INJKMEFK@JVMTI_ERROR_MUST_POSSESS_CAPABI@ 0000000180005ec0     libgetallstktr001.obj
 0002:00000ee8       ??_C@_0BJ@LBFPFPDM@JVMTI_ERROR_NULL_POINTER@ 0000000180005ee8     libgetallstktr001.obj
 0002:00000f08       ??_C@_0BP@CHJPNNEM@JVMTI_ERROR_ABSENT_INFORMATION@ 0000000180005f08     libgetallstktr001.obj
 0002:00000f28       ??_C@_0BP@OMFMNLC@JVMTI_ERROR_INVALID_EVENT_TYPE@ 0000000180005f28     libgetallstktr001.obj
 0002:00000f48       ??_C@_0BN@BIBNPHHO@JVMTI_ERROR_ILLEGAL_ARGUMENT@ 0000000180005f48     libgetallstktr001.obj
 0002:00000f68       ??_C@_0BK@KKNDHDCE@JVMTI_ERROR_NATIVE_METHOD@ 0000000180005f68     libgetallstktr001.obj
 0002:00000f88       ??_C@_0BK@PMKCFHAE@JVMTI_ERROR_OUT_OF_MEMORY@ 0000000180005f88     libgetallstktr001.obj
 0002:00000fa8       ??_C@_0BK@NNJBDMNB@JVMTI_ERROR_ACCESS_DENIED@ 0000000180005fa8     libgetallstktr001.obj
 0002:00000fc8       ??_C@_0BI@GHECLMNC@JVMTI_ERROR_WRONG_PHASE@ 0000000180005fc8     libgetallstktr001.obj
 0002:00000fe0       ??_C@_0BF@OLIHJOII@JVMTI_ERROR_INTERNAL@ 0000000180005fe0     libgetallstktr001.obj
 0002:00000ff8       ??_C@_0BO@EOHGKJHI@JVMTI_ERROR_UNATTACHED_THREAD@ 0000000180005ff8     libgetallstktr001.obj
 0002:00001018       ??_C@_0CA@LKHFDACL@JVMTI_ERROR_INVALID_ENVIRONMENT@ 0000000180006018     libgetallstktr001.obj
 0002:00001038       ??_C@_0BA@MMFHLOKK@?$DMunknown?5error?$DO@ 0000000180006038     libgetallstktr001.obj
 0002:00001048       ??_C@_0CF@CBHOKDB@throwable?5?$DN?5jni?9?$DOExceptionOccur@ 0000000180006048     libgetallstktr001.obj
 0002:00001070       ??_C@_03OFAPEBGM@?$CFs?6@  0000000180006070     libgetallstktr001.obj
 0002:00001078       ??_C@_0DM@LPIGEGNJ@s?2test?2hotspot?2jtreg?2vmTestbase@ 0000000180006078     libgetallstktr001.obj
 0002:000010b8       ??_C@_0CC@NFCNPEPK@Exception?5in?5JNI?5call?5?$CIcleared?$CJ@ 00000001800060b8     libgetallstktr001.obj
 0002:000010e0       ??_C@_0BJ@IBAKFIKF@jni?9?$DOExceptionDescribe?$CI?$CJ@ 00000001800060e0     libgetallstktr001.obj
 0002:00001100       ??_C@_0BG@GGKALKMH@jni?9?$DOExceptionClear?$CI?$CJ@ 0000000180006100     libgetallstktr001.obj
 0002:00001118       ??_C@_0CF@JMGFGJLJ@?$CD?5?5?5verified?5JNI?5assertion?5is?5F@ 0000000180006118     libgetallstktr001.obj
 0002:00001140       ??_C@_0CB@MLNJNCLJ@?5?5jvmti?5error?3?5code?$DN?$CFd?0?5name?$DN?$CFs@ 0000000180006140     libgetallstktr001.obj
 0002:00001168       ??_C@_0CD@OHBGDKMK@?$CD?5?5?5jvmti?5error?3?5code?$DN?$CFd?0?5name?$DN@ 0000000180006168     libgetallstktr001.obj
 0002:00001190       ??_C@_0CG@JNNCGPHB@?$CD?5?5?5error?5expected?3?5code?$DN?$CFd?0?5na@ 0000000180006190     libgetallstktr001.obj
 0002:000011c0       ??_C@_0EB@IMGKPCGE@?$CIstr_obj?5?$DN?5jni?9?$DONewStringUTF?$CIco@ 00000001800061c0     libgetallstktr001.obj
 0002:00001210       ??_C@_0EA@HFOGGBCC@s?2test?2hotspot?2jtreg?2vmTestbase@ 0000000180006210     libgetallstktr001.obj
 0002:00001250       ??_C@_05KKCIMGE@error@     0000000180006250     libgetallstktr001.obj
 0002:00001258       ??_C@_0CJ@JACLEAA@Test?5failed?5by?5setFailStatus?$CI?$CJ?4@ 0000000180006258     libgetallstktr001.obj
 0002:00001290       ??_C@_0EA@PNBCDMOA@s?2test?2hotspot?2jtreg?2vmTestbase@ 0000000180006290     libgetallstktr001.obj
 0002:000012d0       ??_C@_0DI@ILAHDLMP@?$CI?$CKagentThreadProc?$CJ?$CIjvmti_env?0?5a@ 00000001800062d0     libgetallstktr001.obj
 0002:00001308       ??_C@_0BD@KDBALNLB@JVMTI?5agent?5thread@ 0000000180006308     libgetallstktr001.obj
 0002:00001320       ??_C@_0BB@NOKBFPFO@java?1lang?1Thread@ 0000000180006320     libgetallstktr001.obj
 0002:00001334       ??_C@_06FALKBLGB@?$DMinit?$DO@ 0000000180006334     libgetallstktr001.obj
 0002:00001340       ??_C@_0BG@IKDDPPGD@?$CILjava?1lang?1String?$DL?$CJV@ 0000000180006340     libgetallstktr001.obj
 0002:00001360       ??_C@_0EB@IFJBFEKC@?$CIthreadClass?5?$DN?5jni_env?9?$DOFindCla@ 0000000180006360     libgetallstktr001.obj
 0002:000013b0       ??_C@_0GF@FGFIBKKL@?$CIthreadCtor?5?$DN?5jni_env?9?$DOGetMetho@ 00000001800063b0     libgetallstktr001.obj
 0002:00001418       ??_C@_0DN@NCPDJLOG@?$CIthreadName?5?$DN?5jni_env?9?$DONewStrin@ 0000000180006418     libgetallstktr001.obj
 0002:00001460       ??_C@_0FE@PFKODBGC@?$CIthreadObject?5?$DN?5jni_env?9?$DONewObj@ 0000000180006460     libgetallstktr001.obj
 0002:000014c0       ??_C@_0ED@HOBAHHJI@?$CIthreadGlobalRef?5?$DN?5jni_env?9?$DONew@ 00000001800064c0     libgetallstktr001.obj
 0002:00001510       ??_C@_0FN@HNJJAHFC@jvmti_env?9?$DORunAgentThread?$CIagent@ 0000000180006510     libgetallstktr001.obj
 0002:00001570       ??_C@_0EA@MOJDNKDF@Debuggee?5status?5sync?5aborted?5be@ 0000000180006570     libgetallstktr001.obj
 0002:000015b0       ??_C@_0EA@EEOEJAEN@status?5?$DN?5syncDebuggeeStatus?$CIjni@ 00000001800065b0     libgetallstktr001.obj
 0002:000015f0       ??_C@_0BL@JBCFNBMB@nsk_jvmti_resetAgentData?$CI?$CJ@ 00000001800065f0     libgetallstktr001.obj
 0002:00001610       ??_C@_0EL@LPBEELIP@s?2test?2hotspot?2jtreg?2vmTestbase@ 0000000180006610     libgetallstktr001.obj
 0002:00001660       ??_C@_0CK@JDAMFDMJ@jvmti?9?$DOSetTag?$CIo?0?5tag?$CJ?5?$DN?$DN?5JVMTI_@ 0000000180006660     libgetallstktr001.obj
 0002:00001690       ??_C@_0CC@DAMNHKNI@Can?8t?5set?5tag?5?$CFli?5for?5object?5?$CFl@ 0000000180006690     libgetallstktr001.obj
 0002:000016b8       ??_C@_0DL@HAJPNKEF@jvmti?9?$DOGetObjectHashCode?$CIo?0?5?$CGha@ 00000001800066b8     libgetallstktr001.obj
 0002:000016f8       ??_C@_0BL@JFPIEOBF@Can?8t?5get?5hash?5object?5?$CFlx?6@ 00000001800066f8     libgetallstktr001.obj
 0002:00001718       ??_C@_0BG@DICPHBKN@setTag?3?5?$CF08x?5?$DM?9?5?$CF?53li@ 0000000180006718     libgetallstktr001.obj
 0002:00001730       ??_C@_0DH@FCEEBDMJ@?$CIs?5?$DN?5jni?9?$DOGetStringUTFChars?$CIsIn@ 0000000180006730     libgetallstktr001.obj
 0002:00001768       ??_C@_0BJ@OKKGHDCN@Can?8t?5get?5string?5at?5?$CF?$CDp?6@ 0000000180006768     libgetallstktr001.obj
 0002:00001788       ??_C@_0BP@EKFLGGFJ@Can?8t?5get?5string?5at?5?$CF?$CDp?3?5null?6@ 0000000180006788     libgetallstktr001.obj
 0002:000017a8       ??_C@_06ICODBHCL@?5?1?1?5?$CFs@ 00000001800067a8     libgetallstktr001.obj
 0002:000017b0       ??_C@_0DB@KGFPLEGO@?$CIr?5?$DN?5jvmti?9?$DOGetTag?$CIo?0?5?$CGtag?$CJ?$CJ?5?$DN?$DN@ 00000001800067b0     libgetallstktr001.obj
 0002:000017e8       ??_C@_0CO@PDAGBCGJ@Can?8t?5GetTag?5for?5object?5?$CFlx?4?5Re@ 00000001800067e8     libgetallstktr001.obj
 0002:00001818       ??_C@_0CH@HPEODOHC@TEST_BUG?3?5Max?4?5number?5of?5refs?5r@ 0000000180006818     libgetallstktr001.obj
 0002:00001840       ??_C@_0DI@PHFCABIM@?$CIr?5?$DN?5jvmti?9?$DOGetTag?$CIfrom?0?5?$CGtagFr@ 0000000180006840     libgetallstktr001.obj
 0002:00001878       ??_C@_0DI@MDEGFNKD@TEST_BUG?3?5Can?8t?5GetTag?5for?5obje@ 0000000180006878     libgetallstktr001.obj
 0002:000018b0       ??_C@_0DE@MLELJAHM@?$CIr?5?$DN?5jvmti?9?$DOGetTag?$CIto?0?5?$CGtagTo?$CJ?$CJ@ 00000001800068b0     libgetallstktr001.obj
 0002:000018e8       ??_C@_0CJ@KCDEKOCJ@Wrong?5result?5of?5a?5valid?5call?5to@ 00000001800068e8     libgetallstktr001.obj
 0002:00001918       ??_C@_0CI@EDEMEGFA@GetPotentialCapabilities?5return@ 0000000180006918     libgetallstktr001.obj
 0002:00001940       ??_C@_06JBLMLCKL@?$CFs?5?$CFd?6@ 0000000180006940     libgetallstktr001.obj
 0002:00001948       ??_C@_0M@IIAIBNDM@Raw?9monitor@ 0000000180006948     libgetallstktr001.obj
 0002:00001958       ??_C@_0BP@FGJPGNLN@Error?3?5Raw?5monitor?5create?5?$CFd?5?6@ 0000000180006958     libgetallstktr001.obj
 0002:00001978       ??_C@_0BO@OJFPHDDP@Error?3?5Raw?5monitor?5enter?5?$CFd?5?6@ 0000000180006978     libgetallstktr001.obj
 0002:00001998       ??_C@_0BL@GKGBEHOI@Error?3?5RawMonitorExit?5?$CFd?5?6@ 0000000180006998     libgetallstktr001.obj
 0002:000019b8       ??_C@_0DO@PMEMAHNP@FAILED?3?5compare?5frame?3?5thread?5?$CF@ 00000001800069b8     libgetallstktr001.obj
 0002:00001a00       ??_C@_0EA@MMNLDOKP@FAILED?3?5compare?5frame?3?5thread?5?$CF@ 0000000180006a00     libgetallstktr001.obj
 0002:00001a40       ??_C@_0FC@NCMJGAEA@thr?5?$CD?$CFd?3?5compare?5frame?5?$CD?$CFd?3?5fie@ 0000000180006a40     libgetallstktr001.obj
 0002:00001a98       ??_C@_0BA@MGIBPNPB@getallstktr001?9@ 0000000180006a98     libgetallstktr001.obj
 0002:00001aa8       ??_C@_0BP@IMKPCHHJ@compare?5stack?5?$CD?$CFd?3?5thread?3?5?$CFs?6@ 0000000180006aa8     libgetallstktr001.obj
 0002:00001ac8       ??_C@_0CD@ENOIMNMO@compare?5stack?5?$CD?$CFd?3?5thread?5is?5nu@ 0000000180006ac8     libgetallstktr001.obj
 0002:00001af0       ??_C@_0DF@NHCNMNGO@compare?5stack?5?$CD?$CFd?3?5?$CFs?5isn?8t?5tes@ 0000000180006af0     libgetallstktr001.obj
 0002:00001b28       ??_C@_0DP@POBINBGE@FAILED?3?5compare?5stack?5?$CD?$CFd?3?5diff@ 0000000180006b28     libgetallstktr001.obj
 0002:00001b70       ??_C@_0EG@CCBJBCBC@FAILED?3?5compare?5stack?5?$CD?$CFd?3?5diff@ 0000000180006b70     libgetallstktr001.obj
 0002:00001bc0       ??_C@_0FE@PLLAKDBC@compare?5stack?5?$CD?$CFd?3?5fields?5are?5t@ 0000000180006bc0     libgetallstktr001.obj
 0002:00001c18       ??_C@_0BO@LGEFEFHN@Error?3?5GetAllStackTraces?5?$CFd?5?6@ 0000000180006c18     libgetallstktr001.obj
 0002:00001c38       ??_C@_0CC@LBLLBNPM@Error?3?5Allocate?5failed?5with?5?5?$CFd@ 0000000180006c38     libgetallstktr001.obj
 0002:00001c60       ??_C@_0BK@HLILJPBK@Error?3?5GetThreadInfo?5?$CFd?5?6@ 0000000180006c60     libgetallstktr001.obj
 0002:00001c80       ??_C@_0BO@LJFJLPHA@GetThreadInfo?5?$CFd?3?5thread?3?5?$CFs?6@ 0000000180006c80     libgetallstktr001.obj
 0002:00001ca0       ??_C@_0CF@IICFBAAM@Error?3?5GetThreadListStackTraces@ 0000000180006ca0     libgetallstktr001.obj
 0002:00001cc8       ??_C@_0CD@FAOAJHGL@Error?3?5ForceGarbageCollection?5?$CF@ 0000000180006cc8     libgetallstktr001.obj
 0002:00001cf0       ??_C@_0CP@OLJCIGIB@Error?3?5Deallocate?5stack_buf1?5fa@ 0000000180006cf0     libgetallstktr001.obj
 0002:00001d20       ??_C@_0CP@EEDLMLEL@Error?3?5Deallocate?5stack_buf2?5fa@ 0000000180006d20     libgetallstktr001.obj
 0002:00001d50       ??_C@_0DA@NLPCEGIF@Error?3?5Deallocate?5thread_info?5f@ 0000000180006d50     libgetallstktr001.obj
 0002:00001d80       ??_C@_0DA@DBHHJGBG@Error?3?5Deallocate?5thread_list?5f@ 0000000180006d80     libgetallstktr001.obj
 0002:00001dc0       ??_C@_1EC@JIJBPKFM@?$AAa?$AAp?$AAi?$AA?9?$AAm?$AAs?$AA?9?$AAw?$AAi?$AAn?$AA?9?$AAc?$AAo?$AAr?$AAe@ 0000000180006dc0     MSVCRT:thread_safe_statics.obj
 0002:00001e08       ??_C@_1BK@MGMFAEKH@?$AAk?$AAe?$AAr?$AAn?$AAe?$AAl?$AA3?$AA2?$AA?4?$AAd?$AAl?$AAl@ 0000000180006e08     MSVCRT:thread_safe_statics.obj
 0002:00001e28       ??_C@_0BJ@JEBJOJFJ@SleepConditionVariableCS@ 0000000180006e28     MSVCRT:thread_safe_statics.obj
 0002:00001e48       ??_C@_0BJ@PGPPEPCC@WakeAllConditionVariable@ 0000000180006e48     MSVCRT:thread_safe_statics.obj
 0002:00001e68       _pDefaultRawDllMain        0000000180006e68     MSVCRT:dll_dllmain.obj
 0002:00001e68       _pRawDllMain               0000000180006e68     MSVCRT:dll_dllmain.obj
 0002:00001e70       __xmm@ffffffffffffffffffffffffffffffff 0000000180006e70     MSVCRT:utility.obj
 0002:00001e80       _load_config_used          0000000180006e80     MSVCRT:loadcfg.obj
 0002:00002080       _tls_used                  0000000180007080     MSVCRT:tlssup.obj
 0002:000020a8       __volatile_metadata        00000001800070a8     <linker-defined>
 0002:00002468       __rtc_iaa                  0000000180007468     MSVCRT:initsect.obj
 0002:00002470       __rtc_izz                  0000000180007470     MSVCRT:initsect.obj
 0002:00002478       __rtc_taa                  0000000180007478     MSVCRT:initsect.obj
 0002:00002480       __rtc_tzz                  0000000180007480     MSVCRT:initsect.obj
 0002:00002488       _tls_start                 0000000180007488     MSVCRT:tlssup.obj
 0002:0000248c       _Init_thread_epoch         000000018000748c     MSVCRT:thread_safe_statics.obj
 0002:00002490       _tls_end                   0000000180007490     MSVCRT:tlssup.obj
 0002:00002e70       __IMPORT_DESCRIPTOR_KERNEL32 0000000180007e70     kernel32:KERNEL32.dll
 0002:00002e84       __IMPORT_DESCRIPTOR_VCRUNTIME140 0000000180007e84     vcruntime:VCRUNTIME140.dll
 0002:00002e98       __IMPORT_DESCRIPTOR_api-ms-win-crt-runtime-l1-1-0 0000000180007e98     ucrt:api-ms-win-crt-runtime-l1-1-0.dll
 0002:00002eac       __IMPORT_DESCRIPTOR_api-ms-win-crt-stdio-l1-1-0 0000000180007eac     ucrt:api-ms-win-crt-stdio-l1-1-0.dll
 0002:00002ec0       __IMPORT_DESCRIPTOR_api-ms-win-crt-string-l1-1-0 0000000180007ec0     ucrt:api-ms-win-crt-string-l1-1-0.dll
 0002:00002ed4       __NULL_IMPORT_DESCRIPTOR   0000000180007ed4     kernel32:KERNEL32.dll
 0003:00000038       _Init_global_epoch         0000000180009038     MSVCRT:thread_safe_statics.obj
 0003:00000040       __security_cookie          0000000180009040     MSVCRT:gs_cookie.obj
 0003:00000048       __security_cookie_complement 0000000180009048     MSVCRT:gs_cookie.obj
 0003:00000050       __scrt_native_dllmain_reason 0000000180009050     MSVCRT:utility.obj
 0003:00000058       __isa_available            0000000180009058     MSVCRT:cpu_disp.obj
 0003:0000005c       __isa_enabled              000000018000905c     MSVCRT:cpu_disp.obj
 0003:00000060       __memset_fast_string_threshold 0000000180009060     MSVCRT:cpu_disp.obj
 0003:00000068       __memset_nt_threshold      0000000180009068     MSVCRT:cpu_disp.obj
 0003:00000070       __scrt_ucrt_dll_is_in_use  0000000180009070     MSVCRT:ucrt_stubs.obj
 0003:00000080       g_wrongHeapCallbacks       0000000180009080     libgetallstktr001.obj
 0003:00000100       g_szTagInfo                0000000180009100     libgetallstktr001.obj
 0003:00002040       g_tagFlags                 000000018000b040     libgetallstktr001.obj
 0003:00002428       g_refsToVerifyCnt          000000018000b428     libgetallstktr001.obj
 0003:0000242c       g_fakeUserData             000000018000b42c     libgetallstktr001.obj
 0003:00002430       g_tagVisitCount            000000018000b430     libgetallstktr001.obj
 0003:000033d0       g_refsToVerify             000000018000c3d0     libgetallstktr001.obj
 0003:0001aad0       g_userDataError            0000000180023ad0     libgetallstktr001.obj
 0003:0001acb0       ?_OptionsStorage@?1??__local_stdio_printf_options@@9@4_KA 0000000180023cb0     libgetallstktr001.obj
 0003:0001b278       _tls_index                 0000000180024278     MSVCRT:tlssup.obj
 0003:0001b280       __scrt_current_native_startup_state 0000000180024280     MSVCRT:utility.obj
 0003:0001b288       __scrt_native_startup_lock 0000000180024288     MSVCRT:utility.obj
 0003:0001b2c8       __scrt_debugger_hook_flag  00000001800242c8     MSVCRT:utility_desktop.obj
 0003:0001b2d0       ?__type_info_root_node@@3U__type_info_node@@A 00000001800242d0     MSVCRT:tncleanup.obj
 0003:0001b2e0       ?_OptionsStorage@?1??__local_stdio_scanf_options@@9@4_KA 00000001800242e0     MSVCRT:default_local_stdio_options.obj
 0003:0001b2e8       __favor                    00000001800242e8     MSVCRT:cpu_disp.obj
 0003:0001b2f0       __dyn_tls_init_callback    00000001800242f0     <common>

 entry point at        0001:00002800

 Static symbols

 0000:fffd9000       .debug$S                   0000000180000000     getallstktr001.exp
 0000:fffd9000       .debug$S                   0000000180000000     vcruntime:VCRUNTIME140.dll
 0000:fffd9000       .debug$S                   0000000180000000     vcruntime:VCRUNTIME140.dll
 0000:fffd9000       .debug$S                   0000000180000000     vcruntime:VCRUNTIME140.dll
 0000:fffd9000       .debug$S                   0000000180000000     vcruntime:VCRUNTIME140.dll
 0000:fffd9000       .debug$S                   0000000180000000     vcruntime:VCRUNTIME140.dll
 0000:fffd9000       .debug$S                   0000000180000000     vcruntime:VCRUNTIME140.dll
 0000:fffd9000       .debug$S                   0000000180000000     vcruntime:VCRUNTIME140.dll
 0000:fffd9000       .debug$S                   0000000180000000     ucrt:api-ms-win-crt-convert-l1-1-0.dll
 0002:ffffb000       .idata$6                   0000000180000000     ucrt:api-ms-win-crt-convert-l1-1-0.dll
 0000:fffd9000       .debug$S                   0000000180000000     ucrt:api-ms-win-crt-heap-l1-1-0.dll
 0000:fffd9000       .debug$S                   0000000180000000     ucrt:api-ms-win-crt-heap-l1-1-0.dll
 0000:fffd9000       .debug$S                   0000000180000000     ucrt:api-ms-win-crt-heap-l1-1-0.dll
 0000:fffd9000       .debug$S                   0000000180000000     ucrt:api-ms-win-crt-heap-l1-1-0.dll
 0002:ffffb000       .idata$6                   0000000180000000     ucrt:api-ms-win-crt-heap-l1-1-0.dll
 0000:fffd9000       .debug$S                   0000000180000000     ucrt:api-ms-win-crt-runtime-l1-1-0.dll
 0000:fffd9000       .debug$S                   0000000180000000     ucrt:api-ms-win-crt-runtime-l1-1-0.dll
 0000:fffd9000       .debug$S                   0000000180000000     ucrt:api-ms-win-crt-runtime-l1-1-0.dll
 0000:fffd9000       .debug$S                   0000000180000000     ucrt:api-ms-win-crt-runtime-l1-1-0.dll
 0000:fffd9000       .debug$S                   0000000180000000     ucrt:api-ms-win-crt-runtime-l1-1-0.dll
 0000:fffd9000       .debug$S                   0000000180000000     ucrt:api-ms-win-crt-runtime-l1-1-0.dll
 0000:fffd9000       .debug$S                   0000000180000000     ucrt:api-ms-win-crt-runtime-l1-1-0.dll
 0000:fffd9000       .debug$S                   0000000180000000     ucrt:api-ms-win-crt-runtime-l1-1-0.dll
 0000:fffd9000       .debug$S                   0000000180000000     ucrt:api-ms-win-crt-runtime-l1-1-0.dll
 0000:fffd9000       .debug$S                   0000000180000000     ucrt:api-ms-win-crt-runtime-l1-1-0.dll
 0000:fffd9000       .debug$S                   0000000180000000     ucrt:api-ms-win-crt-runtime-l1-1-0.dll
 0000:fffd9000       .debug$S                   0000000180000000     ucrt:api-ms-win-crt-runtime-l1-1-0.dll
 0000:fffd9000       .debug$S                   0000000180000000     ucrt:api-ms-win-crt-runtime-l1-1-0.dll
 0000:fffd9000       .debug$S                   0000000180000000     ucrt:api-ms-win-crt-runtime-l1-1-0.dll
 0000:fffd9000       .debug$S                   0000000180000000     ucrt:api-ms-win-crt-runtime-l1-1-0.dll
 0000:fffd9000       .debug$S                   0000000180000000     ucrt:api-ms-win-crt-runtime-l1-1-0.dll
 0000:fffd9000       .debug$S                   0000000180000000     ucrt:api-ms-win-crt-stdio-l1-1-0.dll
 0000:fffd9000       .debug$S                   0000000180000000     ucrt:api-ms-win-crt-stdio-l1-1-0.dll
 0000:fffd9000       .debug$S                   0000000180000000     ucrt:api-ms-win-crt-stdio-l1-1-0.dll
 0000:fffd9000       .debug$S                   0000000180000000     ucrt:api-ms-win-crt-stdio-l1-1-0.dll
 0000:fffd9000       .debug$S                   0000000180000000     ucrt:api-ms-win-crt-stdio-l1-1-0.dll
 0000:fffd9000       .debug$S                   0000000180000000     ucrt:api-ms-win-crt-stdio-l1-1-0.dll
 0000:fffd9000       .debug$S                   0000000180000000     ucrt:api-ms-win-crt-stdio-l1-1-0.dll
 0000:fffd9000       .debug$S                   0000000180000000     ucrt:api-ms-win-crt-stdio-l1-1-0.dll
 0000:fffd9000       .debug$S                   0000000180000000     ucrt:api-ms-win-crt-stdio-l1-1-0.dll
 0000:fffd9000       .debug$S                   0000000180000000     ucrt:api-ms-win-crt-stdio-l1-1-0.dll
 0000:fffd9000       .debug$S                   0000000180000000     ucrt:api-ms-win-crt-string-l1-1-0.dll
 0000:fffd9000       .debug$S                   0000000180000000     ucrt:api-ms-win-crt-string-l1-1-0.dll
 0000:fffd9000       .debug$S                   0000000180000000     ucrt:api-ms-win-crt-string-l1-1-0.dll
 0000:fffd9000       .debug$S                   0000000180000000     ucrt:api-ms-win-crt-string-l1-1-0.dll
 0000:fffd9000       .debug$S                   0000000180000000     ucrt:api-ms-win-crt-string-l1-1-0.dll
 0000:fffd9000       .debug$S                   0000000180000000     ucrt:api-ms-win-crt-string-l1-1-0.dll
 0000:fffd9000       .debug$S                   0000000180000000     ucrt:api-ms-win-crt-string-l1-1-0.dll
 0000:fffd9000       .debug$S                   0000000180000000     ucrt:api-ms-win-crt-string-l1-1-0.dll
 0000:fffd9000       .debug$S                   0000000180000000     kernel32:KERNEL32.dll
 0000:fffd9000       .debug$S                   0000000180000000     kernel32:KERNEL32.dll
 0000:fffd9000       .debug$S                   0000000180000000     kernel32:KERNEL32.dll
 0000:fffd9000       .debug$S                   0000000180000000     kernel32:KERNEL32.dll
 0000:fffd9000       .debug$S                   0000000180000000     kernel32:KERNEL32.dll
 0000:fffd9000       .debug$S                   0000000180000000     kernel32:KERNEL32.dll
 0000:fffd9000       .debug$S                   0000000180000000     kernel32:KERNEL32.dll
 0000:fffd9000       .debug$S                   0000000180000000     kernel32:KERNEL32.dll
 0000:fffd9000       .debug$S                   0000000180000000     kernel32:KERNEL32.dll
 0000:fffd9000       .debug$S                   0000000180000000     kernel32:KERNEL32.dll
 0000:fffd9000       .debug$S                   0000000180000000     kernel32:KERNEL32.dll
 0000:fffd9000       .debug$S                   0000000180000000     kernel32:KERNEL32.dll
 0000:fffd9000       .debug$S                   0000000180000000     kernel32:KERNEL32.dll
 0000:fffd9000       .debug$S                   0000000180000000     kernel32:KERNEL32.dll
 0000:fffd9000       .debug$S                   0000000180000000     kernel32:KERNEL32.dll
 0000:fffd9000       .debug$S                   0000000180000000     kernel32:KERNEL32.dll
 0000:fffd9000       .debug$S                   0000000180000000     kernel32:KERNEL32.dll
 0000:fffd9000       .debug$S                   0000000180000000     kernel32:KERNEL32.dll
 0000:fffd9000       .debug$S                   0000000180000000     kernel32:KERNEL32.dll
 0000:fffd9000       .debug$S                   0000000180000000     kernel32:KERNEL32.dll
 0000:fffd9000       .debug$S                   0000000180000000     kernel32:KERNEL32.dll
 0000:fffd9000       .debug$S                   0000000180000000     kernel32:KERNEL32.dll
 0000:fffd9000       .debug$S                   0000000180000000     kernel32:KERNEL32.dll
 0000:fffd9000       .debug$S                   0000000180000000     kernel32:KERNEL32.dll
 0000:fffd9000       .debug$S                   0000000180000000     kernel32:KERNEL32.dll
 0000:fffd9000       .debug$S                   0000000180000000     kernel32:KERNEL32.dll
 0000:fffd9000       .debug$S                   0000000180000000     kernel32:KERNEL32.dll
 0000:fffd9000       .debug$S                   0000000180000000     kernel32:KERNEL32.dll
 0001:000011e0       addRefToVerify             00000001800021e0 f   libgetallstktr001.obj
 0001:0000124c       agentThreadWrapper         000000018000224c f   libgetallstktr001.obj
 0001:00001674       file_basename              0000000180002674 f   libgetallstktr001.obj
 0001:00001ce0       startAgentThreadWrapper    0000000180002ce0 f   libgetallstktr001.obj
 0001:00002020       syncDebuggeeStatus         0000000180003020 f   libgetallstktr001.obj
 0001:000022c0       capture_previous_context   00000001800032c0 f   MSVCRT:gs_report.obj
 0001:00002334       ?__scrt_initialize_thread_safe_statics@@YAHXZ 0000000180003334 f   MSVCRT:thread_safe_statics.obj
 0001:00002404       ?__scrt_uninitialize_thread_safe_statics@@YAXXZ 0000000180003404 f   MSVCRT:thread_safe_statics.obj
 0001:000024b0       $$000000                   00000001800034b0     MSVCRT:amdsecgs.obj
 0001:000024e0       ?dllmain_crt_dispatch@@YAHQEAUHINSTANCE__@@KQEAX@Z 00000001800034e0 f   MSVCRT:dll_dllmain.obj
 0001:00002530       ?dllmain_crt_process_attach@@YAHQEAUHINSTANCE__@@QEAX@Z 0000000180003530 f   MSVCRT:dll_dllmain.obj
 0001:00002648       ?dllmain_crt_process_detach@@YAH_N@Z 0000000180003648 f   MSVCRT:dll_dllmain.obj
 0001:000026cc       ?dllmain_dispatch@@YAHQEAUHINSTANCE__@@KQEAX@Z 00000001800036cc f   MSVCRT:dll_dllmain.obj
 0001:000030e0       $$000000                   00000001800040e0     MSVCRT:guard_dispatch.obj
 0001:00003100       $$000000                   0000000180004100     MSVCRT:guard_xfg_dispatch.obj
 0001:00003116       ?fin$0@?0??dllmain_crt_process_attach@@YAHQEAUHINSTANCE__@@QEAX@Z@4HA 0000000180004116 f   MSVCRT:dll_dllmain.obj
 0001:0000312d       ?fin$0@?0??dllmain_crt_process_detach@@YAH_N@Z@4HA 000000018000412d f   MSVCRT:dll_dllmain.obj
 0001:00003146       ?fin$1@?0??dllmain_crt_process_detach@@YAH_N@Z@4HA 0000000180004146 f   MSVCRT:dll_dllmain.obj
 0001:0000315a       ?filt$0@?0??dllmain_dispatch@@YAHQEAUHINSTANCE__@@KQEAX@Z@4HA 000000018000415a f   MSVCRT:dll_dllmain.obj
 0001:00003190       __scrt_is_nonwritable_in_current_image$filt$0 0000000180004190 f   MSVCRT:utility.obj
 0002:000001e8       ?__scrt_initialize_tss_var@@3P6AHXZEA 00000001800051e8     MSVCRT:thread_safe_statics.obj
 0002:00000310       ?opcLengths@@3QBEB         0000000180005310     libgetallstktr001.obj
 0002:00001db0       GS_ExceptionPointers       0000000180006db0     MSVCRT:gs_report.obj
 0002:00002498       $unwind$fprintf            0000000180007498     libgetallstktr001.obj
 0002:000024a4       $unwind$printf             00000001800074a4     libgetallstktr001.obj
 0002:000024b0       $unwind$_snprintf          00000001800074b0     libgetallstktr001.obj
 0002:000024c0       $unwind$?NewObject@JNIEnv_@@QEAAPEAV_jobject@@PEAV_jclass@@PEAU_jmethodID@@ZZ 00000001800074c0     libgetallstktr001.obj
 0002:000024c0       $unwind$nsk_lcomplain      00000001800074c0     libgetallstktr001.obj
 0002:000024c0       $unwind$nsk_ldisplay       00000001800074c0     libgetallstktr001.obj
 0002:000024c8       $unwind$nsk_lvdisplay      00000001800074c8     libgetallstktr001.obj
 0002:000024c8       $unwind$_RTC_Initialize    00000001800074c8     MSVCRT:initsect.obj
 0002:000024c8       $unwind$_RTC_Terminate     00000001800074c8     MSVCRT:initsect.obj
 0002:000024c8       $unwind$?__scrt_initialize_thread_safe_statics@@YAHXZ 00000001800074c8     MSVCRT:thread_safe_statics.obj
 0002:000024d4       $unwind$nsk_lvcomplain     00000001800074d4     libgetallstktr001.obj
 0002:000024ec       $unwind$nsk_ltrace         00000001800074ec     libgetallstktr001.obj
 0002:000024ec       $unwind$__report_gsfailure 00000001800074ec     MSVCRT:gs_report.obj
 0002:000024f4       $unwind$Agent_Initialize   00000001800074f4     libgetallstktr001.obj
 0002:000024f4       $unwind$nsk_lvtrace        00000001800074f4     libgetallstktr001.obj
 0002:000024f4       $unwind$__raise_securityfailure 00000001800074f4     MSVCRT:gs_report.obj
 0002:000024f4       $unwind$__scrt_initialize_crt 00000001800074f4     MSVCRT:utility.obj
 0002:000024f4       $unwind$__scrt_initialize_onexit_tables 00000001800074f4     MSVCRT:utility.obj
 0002:000024f4       $unwind$__scrt_release_startup_lock 00000001800074f4     MSVCRT:utility.obj
 0002:000024f4       $unwind$__scrt_uninitialize_crt 00000001800074f4     MSVCRT:utility.obj
 0002:000024f4       $unwind$_onexit            00000001800074f4     MSVCRT:utility.obj
 0002:000024fc       $unwind$nsk_lverify        00000001800074fc     libgetallstktr001.obj
 0002:0000250c       $unwind$nsk_vprintf        000000018000750c     libgetallstktr001.obj
 0002:0000251c       $unwind$nsk_printf         000000018000751c     libgetallstktr001.obj
 0002:00002524       $unwind$?nsk_jni_lverify@@YAHHPEAUJNIEnv_@@HQEBDH1ZZ 0000000180007524     libgetallstktr001.obj
 0002:00002538       $unwind$?nsk_jni_check_exception@@YAHPEAUJNIEnv_@@QEBDH@Z 0000000180007538     libgetallstktr001.obj
 0002:00002554       $unwind$Java_nsk_jvmti_unit_FollowReferences_FollowRefObjects_resetTags 0000000180007554     libgetallstktr001.obj
 0002:00002554       $unwind$Java_nsk_jvmti_unit_GetAllStackTraces_getallstktr001_DeallocateBuffers 0000000180007554     libgetallstktr001.obj
 0002:00002554       $unwind$Java_nsk_jvmti_unit_GetAllStackTraces_getallstktr001_ForceGC 0000000180007554     libgetallstktr001.obj
 0002:00002554       $unwind$Java_nsk_jvmti_unit_GetAllStackTraces_getallstktr001_RawMonitorEnter 0000000180007554     libgetallstktr001.obj
 0002:00002554       $unwind$Java_nsk_jvmti_unit_GetAllStackTraces_getallstktr001_RawMonitorExit 0000000180007554     libgetallstktr001.obj
 0002:00002554       $unwind$addRefToVerify     0000000180007554     libgetallstktr001.obj
 0002:00002554       $unwind$nsk_jvmti_resetAgentData 0000000180007554     libgetallstktr001.obj
 0002:00002554       $unwind$nsk_jvmti_setFailStatus 0000000180007554     libgetallstktr001.obj
 0002:00002554       $unwind$__scrt_initialize_default_local_stdio_options 0000000180007554     MSVCRT:default_local_stdio_options.obj
 0002:00002554       $unwind$?dllmain_crt_dispatch@@YAHQEAUHINSTANCE__@@KQEAX@Z 0000000180007554     MSVCRT:dll_dllmain.obj
 0002:00002554       $unwind$DllMain            0000000180007554     MSVCRT:dll_dllmain_stub.obj
 0002:00002554       $unwind$__GSHandlerCheck   0000000180007554     MSVCRT:gshandler.obj
 0002:00002554       $unwind$?__scrt_uninitialize_thread_safe_statics@@YAXXZ 0000000180007554     MSVCRT:thread_safe_statics.obj
 0002:00002554       $unwind$__scrt_acquire_startup_lock 0000000180007554     MSVCRT:utility.obj
 0002:00002554       $unwind$__scrt_dllmain_after_initialize_c 0000000180007554     MSVCRT:utility.obj
 0002:00002554       $unwind$__scrt_dllmain_before_initialize_c 0000000180007554     MSVCRT:utility.obj
 0002:00002554       $unwind$__scrt_dllmain_crt_thread_attach 0000000180007554     MSVCRT:utility.obj
 0002:00002554       $unwind$__scrt_dllmain_crt_thread_detach 0000000180007554     MSVCRT:utility.obj
 0002:00002554       $unwind$__scrt_dllmain_uninitialize_c 0000000180007554     MSVCRT:utility.obj
 0002:00002554       $unwind$__scrt_dllmain_uninitialize_critical 0000000180007554     MSVCRT:utility.obj
 0002:00002554       $unwind$atexit             0000000180007554     MSVCRT:utility.obj
 0002:0000255c       $unwind$nsk_jvmti_lverify  000000018000755c     libgetallstktr001.obj
 0002:00002570       $unwind$exitOnError        0000000180007570     libgetallstktr001.obj
 0002:00002580       $unwind$Java_nsk_share_jvmti_ArgumentHandler_getAgentOptionsString 0000000180007580     libgetallstktr001.obj
 0002:00002594       $unwind$Java_nsk_jvmti_unit_FollowReferences_FollowRefObjects_getTag 0000000180007594     libgetallstktr001.obj
 0002:00002594       $unwind$Java_nsk_share_jvmti_DebugeeClass_checkStatus 0000000180007594     libgetallstktr001.obj
 0002:00002594       $unwind$agentThreadWrapper 0000000180007594     libgetallstktr001.obj
 0002:000025a4       $unwind$startAgentThreadWrapper 00000001800075a4     libgetallstktr001.obj
 0002:000025c0       $unwind$syncDebuggeeStatus 00000001800075c0     libgetallstktr001.obj
 0002:000025c0       $unwind$__scrt_dllmain_exception_filter 00000001800075c0     MSVCRT:utility.obj
 0002:000025d4       $unwind$Java_nsk_share_jvmti_DebugeeClass_resetAgentData 00000001800075d4     libgetallstktr001.obj
 0002:000025dc       $unwind$MA_checkStatus     00000001800075dc     libgetallstktr001.obj
 0002:000025f0       $unwind$Java_nsk_jvmti_unit_FollowReferences_FollowRefObjects_setTag 00000001800075f0     libgetallstktr001.obj
 0002:00002608       $unwind$Java_nsk_jvmti_unit_FollowReferences_FollowRefObjects_addRefToVerify 0000000180007608     libgetallstktr001.obj
 0002:00002624       $unwind$Java_nsk_jvmti_unit_GetAllStackTraces_getallstktr001_CreateRawMonitor 0000000180007624     libgetallstktr001.obj
 0002:00002634       $unwind$compare_all_frames 0000000180007634     libgetallstktr001.obj
 0002:0000264c       $unwind$compare_one_stack_trace 000000018000764c     libgetallstktr001.obj
 0002:00002664       $unwind$compare_all_stack_traces 0000000180007664     libgetallstktr001.obj
 0002:0000267c       $unwind$Java_nsk_jvmti_unit_GetAllStackTraces_getallstktr001_GetAllStackTraces 000000018000767c     libgetallstktr001.obj
 0002:00002690       $unwind$Java_nsk_jvmti_unit_GetAllStackTraces_getallstktr001_GetThreadsInfo 0000000180007690     libgetallstktr001.obj
 0002:00002690       $unwind$_DllMainCRTStartup 0000000180007690     MSVCRT:dll_dllmain.obj
 0002:000026a0       $unwind$Java_nsk_jvmti_unit_GetAllStackTraces_getallstktr001_GetThreadListStackTraces 00000001800076a0     libgetallstktr001.obj
 0002:000026a8       $unwind$capture_previous_context 00000001800076a8     MSVCRT:gs_report.obj
 0002:000026b4       $unwind$__GSHandlerCheckCommon 00000001800076b4     MSVCRT:gshandler.obj
 0002:000026c0       $xdatasym                  00000001800076c0     MSVCRT:amdsecgs.obj
 0002:000026c4       $unwind$?dllmain_crt_process_attach@@YAHQEAUHINSTANCE__@@QEAX@Z 00000001800076c4     MSVCRT:dll_dllmain.obj
 0002:00002700       $unwind$?fin$0@?0??dllmain_crt_process_attach@@YAHQEAUHINSTANCE__@@QEAX@Z@4HA 0000000180007700     MSVCRT:dll_dllmain.obj
 0002:00002700       $unwind$?fin$0@?0??dllmain_crt_process_detach@@YAH_N@Z@4HA 0000000180007700     MSVCRT:dll_dllmain.obj
 0002:00002700       $unwind$?fin$1@?0??dllmain_crt_process_detach@@YAH_N@Z@4HA 0000000180007700     MSVCRT:dll_dllmain.obj
 0002:00002708       $unwind$?dllmain_crt_process_detach@@YAH_N@Z 0000000180007708     MSVCRT:dll_dllmain.obj
 0002:0000275c       $unwind$?dllmain_dispatch@@YAHQEAUHINSTANCE__@@KQEAX@Z 000000018000775c     MSVCRT:dll_dllmain.obj
 0002:00002784       $unwind$?filt$0@?0??dllmain_dispatch@@YAHQEAUHINSTANCE__@@KQEAX@Z@4HA 0000000180007784     MSVCRT:dll_dllmain.obj
 0002:0000278c       $unwind$__scrt_is_nonwritable_in_current_image 000000018000778c     MSVCRT:utility.obj
 0002:000027ac       $unwind$__scrt_is_nonwritable_in_current_image$filt$0 00000001800077ac     MSVCRT:utility.obj
 0002:000027b4       $unwind$__scrt_fastfail    00000001800077b4     MSVCRT:utility_desktop.obj
 0002:000027c4       $unwind$__security_init_cookie 00000001800077c4     MSVCRT:gs_support.obj
 0002:000027d0       $unwind$__isa_available_init 00000001800077d0     MSVCRT:cpu_disp.obj
 0002:000027e0       $xdatasym                  00000001800077e0     MSVCRT:guard_dispatch.obj
 0002:000027e8       $xdatasym                  00000001800077e8     MSVCRT:guard_xfg_dispatch.obj
 0002:000027f0       .edata                     00000001800077f0     getallstktr001.exp
 0002:00002818       rgpv                       0000000180007818     getallstktr001.exp
 0002:00002878       rgszName                   0000000180007878     getallstktr001.exp
 0002:000028d8       rgwOrd                     00000001800078d8     getallstktr001.exp
 0002:00002908       szName                     0000000180007908     getallstktr001.exp
 0002:0000291b       $N00001                    000000018000791b     getallstktr001.exp
 0002:0000292a       $N00002                    000000018000792a     getallstktr001.exp
 0002:00002937       $N00003                    0000000180007937     getallstktr001.exp
 0002:0000297c       $N00004                    000000018000797c     getallstktr001.exp
 0002:000029b9       $N00005                    00000001800079b9     getallstktr001.exp
 0002:00002a01       $N00006                    0000000180007a01     getallstktr001.exp
 0002:00002a41       $N00007                    0000000180007a41     getallstktr001.exp
 0002:00002a7e       $N00008                    0000000180007a7e     getallstktr001.exp
 0002:00002ac6       $N00009                    0000000180007ac6     getallstktr001.exp
 0002:00002b0c       $N00010                    0000000180007b0c     getallstktr001.exp
 0002:00002b53       $N00011                    0000000180007b53     getallstktr001.exp
 0002:00002b90       $N00012                    0000000180007b90     getallstktr001.exp
 0002:00002bd7       $N00013                    0000000180007bd7     getallstktr001.exp
 0002:00002c16       $N00014                    0000000180007c16     getallstktr001.exp
 0002:00002c64       $N00015                    0000000180007c64     getallstktr001.exp
 0002:00002ca8       $N00016                    0000000180007ca8     getallstktr001.exp
 0002:00002ced       $N00017                    0000000180007ced     getallstktr001.exp
 0002:00002d31       $N00018                    0000000180007d31     getallstktr001.exp
 0002:00002d6c       $N00019                    0000000180007d6c     getallstktr001.exp
 0002:00002d9a       $N00020                    0000000180007d9a     getallstktr001.exp
 0002:00002dcb       $N00021                    0000000180007dcb     getallstktr001.exp
 0002:00002dfa       $N00022                    0000000180007dfa     getallstktr001.exp
 0002:00002e29       $N00023                    0000000180007e29     getallstktr001.exp
 0002:00002e5e       $N00024                    0000000180007e5e     getallstktr001.exp
 0002:0000326a       .idata$6                   000000018000826a     kernel32:KERNEL32.dll
 0002:000032ce       .idata$6                   00000001800082ce     vcruntime:VCRUNTIME140.dll
 0002:0000343a       .idata$6                   000000018000843a     ucrt:api-ms-win-crt-runtime-l1-1-0.dll
 0002:0000345c       .idata$6                   000000018000845c     ucrt:api-ms-win-crt-stdio-l1-1-0.dll
 0002:0000347c       .idata$6                   000000018000847c     ucrt:api-ms-win-crt-string-l1-1-0.dll
 0003:00000000       ?codeAttributeName@@3PEBDEB 0000000180009000     libgetallstktr001.obj
 0003:00000008       ?lineNumberAttributeName@@3PEBDEB 0000000180009008     libgetallstktr001.obj
 0003:00000010       ?localVarAttributeName@@3PEBDEB 0000000180009010     libgetallstktr001.obj
 0003:00000018       ?localVarTypeAttributeName@@3PEBDEB 0000000180009018     libgetallstktr001.obj
 0003:00000020       ?stackMapAttributeName@@3PEBDEB 0000000180009020     libgetallstktr001.obj
 0003:00000028       ?callBytes@@3PAEA          0000000180009028     libgetallstktr001.obj
 0003:0000002c       ?allocBytes@@3PAEA         000000018000902c     libgetallstktr001.obj
 0003:00000030       ?TEST_THREAD_NAME_PREFIX@?1??compare_one_stack_trace@@9@4PEBDEB 0000000180009030     libgetallstktr001.obj
 0003:0001aad4       redefineAttempted          0000000180023ad4     libgetallstktr001.obj
 0003:0001aad8       nsk_context                0000000180023ad8     libgetallstktr001.obj
 0003:0001aae4       redefineSucceed            0000000180023ae4     libgetallstktr001.obj
 0003:0001aae8       agentFailed                0000000180023ae8     libgetallstktr001.obj
 0003:0001aaec       currentAgentStatus         0000000180023aec     libgetallstktr001.obj
 0003:0001aaf0       context                    0000000180023af0     libgetallstktr001.obj
 0003:0001aba8       agentThread                0000000180023ba8     libgetallstktr001.obj
 0003:0001abb0       agentThreadProc            0000000180023bb0     libgetallstktr001.obj
 0003:0001abb8       agentThreadArg             0000000180023bb8     libgetallstktr001.obj
 0003:0001abc0       agent_data                 0000000180023bc0     libgetallstktr001.obj
 0003:0001abd0       jvmti_env                  0000000180023bd0     libgetallstktr001.obj
 0003:0001abd8       jvm                        0000000180023bd8     libgetallstktr001.obj
 0003:0001abe0       jni_env                    0000000180023be0     libgetallstktr001.obj
 0003:0001abe8       checkStatus_func           0000000180023be8     libgetallstktr001.obj
 0003:0001abf0       ?codeAttributeIndex@@3GA   0000000180023bf0     libgetallstktr001.obj
 0003:0001abf4       ?lineNumberAttributeIndex@@3GA 0000000180023bf4     libgetallstktr001.obj
 0003:0001abf8       ?localVarAttributeIndex@@3GA 0000000180023bf8     libgetallstktr001.obj
 0003:0001abfc       ?localVarTypeAttributeIndex@@3GA 0000000180023bfc     libgetallstktr001.obj
 0003:0001ac00       ?stackMapAttributeIndex@@3GA 0000000180023c00     libgetallstktr001.obj
 0003:0001ac04       ?stackFrameOffset@@3GA     0000000180023c04     libgetallstktr001.obj
 0003:0001ac08       ?mode@@3HA                 0000000180023c08     libgetallstktr001.obj
 0003:0001ac0c       ?constantPoolSize@@3GA     0000000180023c0c     libgetallstktr001.obj
 0003:0001ac10       ?orig@@3PEBEEB             0000000180023c10     libgetallstktr001.obj
 0003:0001ac18       ?gen@@3PEAEEA              0000000180023c18     libgetallstktr001.obj
 0003:0001ac20       ?inputPos@@3PEAEEA         0000000180023c20     libgetallstktr001.obj
 0003:0001ac28       ?endPos@@3PEBEEB           0000000180023c28     libgetallstktr001.obj
 0003:0001ac30       ?genPos@@3PEAEEA           0000000180023c30     libgetallstktr001.obj
 0003:0001ac38       ?markPos@@3PEAEEA          0000000180023c38     libgetallstktr001.obj
 0003:0001ac40       ?constantPool@@3PEAPEADEA  0000000180023c40     libgetallstktr001.obj
 0003:0001ac48       ?constantPoolCount@@3GA    0000000180023c48     libgetallstktr001.obj
 0003:0001ac4c       ?zeroBytes@@3PAEA          0000000180023c4c     libgetallstktr001.obj
 0003:0001ac50       ?codeLength@@3IA           0000000180023c50     libgetallstktr001.obj
 0003:0001ac54       iGlobalStatus              0000000180023c54     libgetallstktr001.obj
 0003:0001ac58       ?map@@3PEAIEA              0000000180023c58     libgetallstktr001.obj
 0003:0001ac60       ?widening@@3PEACEA         0000000180023c60     libgetallstktr001.obj
 0003:0001ac68       jvmti                      0000000180023c68     libgetallstktr001.obj
 0003:0001ac70       jvmti_caps                 0000000180023c70     libgetallstktr001.obj
 0003:0001ac80       jraw_monitor               0000000180023c80     libgetallstktr001.obj
 0003:0001ac88       stack_buf1                 0000000180023c88     libgetallstktr001.obj
 0003:0001ac90       stack_buf2                 0000000180023c90     libgetallstktr001.obj
 0003:0001ac98       thread_list                0000000180023c98     libgetallstktr001.obj
 0003:0001aca0       thread_info                0000000180023ca0     libgetallstktr001.obj
 0003:0001aca8       threads_count              0000000180023ca8     libgetallstktr001.obj
 0003:0001acc0       GS_ExceptionRecord         0000000180023cc0     MSVCRT:gs_report.obj
 0003:0001ad60       GS_ContextRecord           0000000180023d60     MSVCRT:gs_report.obj
 0003:0001b230       ?g_tss_cv@@3U_RTL_CONDITION_VARIABLE@@A 0000000180024230     MSVCRT:thread_safe_statics.obj
 0003:0001b238       ?g_tss_event@@3PEAXEA      0000000180024238     MSVCRT:thread_safe_statics.obj
 0003:0001b240       ?g_tss_mutex@@3U_RTL_CRITICAL_SECTION@@A 0000000180024240     MSVCRT:thread_safe_statics.obj
 0003:0001b268       ?g_sleep_condition_variable_cs@@3P6AHPEAU_RTL_CONDITION_VARIABLE@@PEAU_RTL_CRITICAL_SECTION@@K@ZEA 0000000180024268     MSVCRT:thread_safe_statics.obj
 0003:0001b270       ?g_wake_all_condition_variable@@3P6AXPEAU_RTL_CONDITION_VARIABLE@@@ZEA 0000000180024270     MSVCRT:thread_safe_statics.obj
 0003:0001b27c       ?__proc_attached@@3HA      000000018002427c     MSVCRT:dll_dllmain.obj
 0003:0001b290       ?is_initialized_as_dll@@3_NA 0000000180024290     MSVCRT:utility.obj
 0003:0001b291       ?module_local_atexit_table_initialized@@3_NA 0000000180024291     MSVCRT:utility.obj
 0003:0001b298       ?module_local_atexit_table@@3U_onexit_table_t@@A 0000000180024298     MSVCRT:utility.obj
 0003:0001b2b0       ?module_local_at_quick_exit_table@@3U_onexit_table_t@@A 00000001800242b0     MSVCRT:utility.obj
